###############################################################################
#
# IAR ELF Linker V7.50.2.10312/W32 for ARM                02/Jun/2020  20:26:00
# Copyright 2007-2015 IAR Systems AB.
#
#    Output file  =  
#        D:\Projects\MicroTechnics\Projects_site\MT_I2C_Example\EWARM\MT_I2C_Example\Exe\MT_I2C_Example.out
#    Map file     =  
#        D:\Projects\MicroTechnics\Projects_site\MT_I2C_Example\EWARM\MT_I2C_Example\List\MT_I2C_Example.map
#    Command line =  
#        D:\Projects\MicroTechnics\Projects_site\MT_I2C_Example\EWARM\MT_I2C_Example\Obj\main.o
#        D:\Projects\MicroTechnics\Projects_site\MT_I2C_Example\EWARM\MT_I2C_Example\Obj\startup_stm32f103xe.o
#        D:\Projects\MicroTechnics\Projects_site\MT_I2C_Example\EWARM\MT_I2C_Example\Obj\stm32f1xx_hal.o
#        D:\Projects\MicroTechnics\Projects_site\MT_I2C_Example\EWARM\MT_I2C_Example\Obj\stm32f1xx_hal_cortex.o
#        D:\Projects\MicroTechnics\Projects_site\MT_I2C_Example\EWARM\MT_I2C_Example\Obj\stm32f1xx_hal_dma.o
#        D:\Projects\MicroTechnics\Projects_site\MT_I2C_Example\EWARM\MT_I2C_Example\Obj\stm32f1xx_hal_exti.o
#        D:\Projects\MicroTechnics\Projects_site\MT_I2C_Example\EWARM\MT_I2C_Example\Obj\stm32f1xx_hal_flash.o
#        D:\Projects\MicroTechnics\Projects_site\MT_I2C_Example\EWARM\MT_I2C_Example\Obj\stm32f1xx_hal_flash_ex.o
#        D:\Projects\MicroTechnics\Projects_site\MT_I2C_Example\EWARM\MT_I2C_Example\Obj\stm32f1xx_hal_gpio.o
#        D:\Projects\MicroTechnics\Projects_site\MT_I2C_Example\EWARM\MT_I2C_Example\Obj\stm32f1xx_hal_gpio_ex.o
#        D:\Projects\MicroTechnics\Projects_site\MT_I2C_Example\EWARM\MT_I2C_Example\Obj\stm32f1xx_hal_i2c.o
#        D:\Projects\MicroTechnics\Projects_site\MT_I2C_Example\EWARM\MT_I2C_Example\Obj\stm32f1xx_hal_msp.o
#        D:\Projects\MicroTechnics\Projects_site\MT_I2C_Example\EWARM\MT_I2C_Example\Obj\stm32f1xx_hal_pwr.o
#        D:\Projects\MicroTechnics\Projects_site\MT_I2C_Example\EWARM\MT_I2C_Example\Obj\stm32f1xx_hal_rcc.o
#        D:\Projects\MicroTechnics\Projects_site\MT_I2C_Example\EWARM\MT_I2C_Example\Obj\stm32f1xx_hal_rcc_ex.o
#        D:\Projects\MicroTechnics\Projects_site\MT_I2C_Example\EWARM\MT_I2C_Example\Obj\stm32f1xx_hal_tim.o
#        D:\Projects\MicroTechnics\Projects_site\MT_I2C_Example\EWARM\MT_I2C_Example\Obj\stm32f1xx_hal_tim_ex.o
#        D:\Projects\MicroTechnics\Projects_site\MT_I2C_Example\EWARM\MT_I2C_Example\Obj\stm32f1xx_it.o
#        D:\Projects\MicroTechnics\Projects_site\MT_I2C_Example\EWARM\MT_I2C_Example\Obj\system_stm32f1xx.o
#        --redirect _Printf=_PrintfFull --redirect _Scanf=_ScanfFull -o
#        D:\Projects\MicroTechnics\Projects_site\MT_I2C_Example\EWARM\MT_I2C_Example\Exe\MT_I2C_Example.out
#        --map
#        D:\Projects\MicroTechnics\Projects_site\MT_I2C_Example\EWARM\MT_I2C_Example\List\MT_I2C_Example.map
#        --config
#        D:\Projects\MicroTechnics\Projects_site\MT_I2C_Example\EWARM/stm32f103xe_flash.icf
#        --semihosting --entry __iar_program_start --vfe
#
###############################################################################

*******************************************************************************
*** RUNTIME MODEL ATTRIBUTES
***

CppFlavor       = *
__SystemLibrary = DLib


*******************************************************************************
*** PLACEMENT SUMMARY
***

"A1":  place at 0x08000000 { ro section .intvec };
"P1":  place in [from 0x08000000 to 0x0807ffff] { ro };
"P2":  place in [from 0x20000000 to 0x2000ffff] { rw, block CSTACK, block HEAP };

  Section            Kind        Address    Size  Object
  -------            ----        -------    ----  ------
"A1":                                      0x130
  .intvec            ro code  0x08000000   0x130  startup_stm32f103xe.o [1]
                            - 0x08000130   0x130

"P1":                                     0x2640
  .text              ro code  0x08000130  0x12e0  stm32f1xx_hal_i2c.o [1]
  .text              ro code  0x08001410    0xf0  stm32f1xx_hal_msp.o [1]
  .text              ro code  0x08001500   0x6f0  stm32f1xx_hal_rcc.o [1]
  .text              ro code  0x08001bf0   0x134  main.o [1]
  .text              ro code  0x08001d24   0x1fe  stm32f1xx_hal_dma.o [1]
  .rodata            const    0x08001f22     0x2  stm32f1xx_hal_rcc.o [1]
  .text              ro code  0x08001f24     0x6  ABImemclr4.o [4]
  .text              ro code  0x08001f2c   0x31c  stm32f1xx_hal_gpio.o [1]
  .text              ro code  0x08002248   0x144  stm32f1xx_hal_cortex.o [1]
  .text              ro code  0x0800238c    0x8c  stm32f1xx_hal.o [1]
  .text              ro code  0x08002418    0x56  ABImemcpy_unaligned.o [4]
  .text              ro code  0x08002470    0x32  ABImemset48.o [4]
  .text              ro code  0x080024a4    0x68  system_stm32f1xx.o [1]
  .text              ro code  0x0800250c    0x40  zero_init3.o [4]
  .text              ro code  0x0800254c    0x30  stm32f1xx_it.o [1]
  .text              ro code  0x0800257c    0x2c  copy_init3.o [4]
  .text              ro code  0x080025a8    0x28  data_init.o [4]
  .iar.init_table    const    0x080025d0    0x24  - Linker created -
  .text              ro code  0x080025f4    0x1a  cmain.o [4]
  .text              ro code  0x0800260e     0x4  low_level_init.o [3]
  .text              ro code  0x08002612     0x4  exit.o [3]
  .text              ro code  0x08002618     0xa  cexit.o [4]
  .text              ro code  0x08002624    0x14  exit.o [5]
  .rodata            const    0x08002638    0x10  stm32f1xx_hal_rcc.o [1]
  .rodata            const    0x08002648    0x10  system_stm32f1xx.o [1]
  .text              ro code  0x08002658    0x10  startup_stm32f103xe.o [1]
  .text              ro code  0x08002668     0xc  cstartup_M.o [4]
  Initializer bytes  const    0x08002674     0xc  <for P2-1>
  .rodata            const    0x08002680     0x8  system_stm32f1xx.o [1]
  .text              ro code  0x08002688     0x4  startup_stm32f103xe.o [1]
  .text              ro code  0x0800268c     0x4  startup_stm32f103xe.o [1]
  .text              ro code  0x08002690     0x4  startup_stm32f103xe.o [1]
  .text              ro code  0x08002694     0x4  startup_stm32f103xe.o [1]
  .text              ro code  0x08002698     0x4  startup_stm32f103xe.o [1]
  .text              ro code  0x0800269c     0x4  startup_stm32f103xe.o [1]
  .text              ro code  0x080026a0     0x4  startup_stm32f103xe.o [1]
  .text              ro code  0x080026a4     0x4  startup_stm32f103xe.o [1]
  .text              ro code  0x080026a8     0x4  startup_stm32f103xe.o [1]
  .text              ro code  0x080026ac     0x4  startup_stm32f103xe.o [1]
  .text              ro code  0x080026b0     0x4  startup_stm32f103xe.o [1]
  .text              ro code  0x080026b4     0x4  startup_stm32f103xe.o [1]
  .text              ro code  0x080026b8     0x4  startup_stm32f103xe.o [1]
  .text              ro code  0x080026bc     0x4  startup_stm32f103xe.o [1]
  .text              ro code  0x080026c0     0x4  startup_stm32f103xe.o [1]
  .text              ro code  0x080026c4     0x4  startup_stm32f103xe.o [1]
  .text              ro code  0x080026c8     0x4  startup_stm32f103xe.o [1]
  .text              ro code  0x080026cc     0x4  startup_stm32f103xe.o [1]
  .text              ro code  0x080026d0     0x4  startup_stm32f103xe.o [1]
  .text              ro code  0x080026d4     0x4  startup_stm32f103xe.o [1]
  .text              ro code  0x080026d8     0x4  startup_stm32f103xe.o [1]
  .text              ro code  0x080026dc     0x4  startup_stm32f103xe.o [1]
  .text              ro code  0x080026e0     0x4  startup_stm32f103xe.o [1]
  .text              ro code  0x080026e4     0x4  startup_stm32f103xe.o [1]
  .text              ro code  0x080026e8     0x4  startup_stm32f103xe.o [1]
  .text              ro code  0x080026ec     0x4  startup_stm32f103xe.o [1]
  .text              ro code  0x080026f0     0x4  startup_stm32f103xe.o [1]
  .text              ro code  0x080026f4     0x4  startup_stm32f103xe.o [1]
  .text              ro code  0x080026f8     0x4  startup_stm32f103xe.o [1]
  .text              ro code  0x080026fc     0x4  startup_stm32f103xe.o [1]
  .text              ro code  0x08002700     0x4  startup_stm32f103xe.o [1]
  .text              ro code  0x08002704     0x4  startup_stm32f103xe.o [1]
  .text              ro code  0x08002708     0x4  startup_stm32f103xe.o [1]
  .text              ro code  0x0800270c     0x4  startup_stm32f103xe.o [1]
  .text              ro code  0x08002710     0x4  startup_stm32f103xe.o [1]
  .text              ro code  0x08002714     0x4  startup_stm32f103xe.o [1]
  .text              ro code  0x08002718     0x4  startup_stm32f103xe.o [1]
  .text              ro code  0x0800271c     0x4  startup_stm32f103xe.o [1]
  .text              ro code  0x08002720     0x4  startup_stm32f103xe.o [1]
  .text              ro code  0x08002724     0x4  startup_stm32f103xe.o [1]
  .text              ro code  0x08002728     0x4  startup_stm32f103xe.o [1]
  .text              ro code  0x0800272c     0x4  startup_stm32f103xe.o [1]
  .text              ro code  0x08002730     0x4  startup_stm32f103xe.o [1]
  .text              ro code  0x08002734     0x4  startup_stm32f103xe.o [1]
  .text              ro code  0x08002738     0x4  startup_stm32f103xe.o [1]
  .text              ro code  0x0800273c     0x4  startup_stm32f103xe.o [1]
  .text              ro code  0x08002740     0x4  startup_stm32f103xe.o [1]
  .text              ro code  0x08002744     0x4  startup_stm32f103xe.o [1]
  .text              ro code  0x08002748     0x4  startup_stm32f103xe.o [1]
  .text              ro code  0x0800274c     0x4  startup_stm32f103xe.o [1]
  .text              ro code  0x08002750     0x4  startup_stm32f103xe.o [1]
  .text              ro code  0x08002754     0x4  startup_stm32f103xe.o [1]
  .text              ro code  0x08002758     0x4  startup_stm32f103xe.o [1]
  .text              ro code  0x0800275c     0x4  startup_stm32f103xe.o [1]
  .text              ro code  0x08002760     0x4  startup_stm32f103xe.o [1]
  .text              ro code  0x08002764     0x4  startup_stm32f103xe.o [1]
  .text              ro code  0x08002768     0x4  startup_stm32f103xe.o [1]
  .text              ro code  0x0800276c     0x4  startup_stm32f103xe.o [1]
  .rodata            const    0x08002770     0x0  zero_init3.o [4]
  .rodata            const    0x08002770     0x0  copy_init3.o [4]
                            - 0x08002770  0x2640

"P2", part 1 of 3:                           0xc
  P2-1                        0x20000000     0xa  <Init block>
    .data            inited   0x20000000     0x4  stm32f1xx_hal.o [1]
    .data            inited   0x20000004     0x4  system_stm32f1xx.o [1]
    .data            inited   0x20000008     0x1  main.o [1]
    .data            inited   0x20000009     0x1  stm32f1xx_hal.o [1]
                            - 0x2000000a     0xa

"P2", part 2 of 3:                         0x400
  CSTACK                      0x20000010   0x400  <Block>
    CSTACK           uninit   0x20000010   0x400  <Block tail>
                            - 0x20000410   0x400

"P2", part 3 of 3:                          0x5c
  .bss               zero     0x20000410    0x54  main.o [1]
  .bss               zero     0x20000464     0x4  stm32f1xx_hal.o [1]
  .bss               zero     0x20000468     0x1  main.o [1]
                            - 0x20000469    0x59


*******************************************************************************
*** INIT TABLE
***

          Address     Size
          -------     ----
Zero (__iar_zero_init3)
    1 destination range, total size 0x59:
          0x20000410  0x59

Copy (__iar_copy_init3)
    1 source range, total size 0xc (120% of destination):
          0x08002674   0xc
    1 destination range, total size 0xa:
          0x20000000   0xa



*******************************************************************************
*** MODULE SUMMARY
***

    Module                  ro code  ro data  rw data
    ------                  -------  -------  -------
D:\Projects\MicroTechnics\Projects_site\MT_I2C_Example\EWARM\MT_I2C_Example\Obj: [1]
    main.o                      308        1       86
    startup_stm32f103xe.o       552
    stm32f1xx_hal.o             140        5        9
    stm32f1xx_hal_cortex.o      324
    stm32f1xx_hal_dma.o         510
    stm32f1xx_hal_gpio.o        796
    stm32f1xx_hal_i2c.o       4 832
    stm32f1xx_hal_msp.o         240
    stm32f1xx_hal_rcc.o       1 776       18
    stm32f1xx_it.o               48
    system_stm32f1xx.o          104       28        4
    -------------------------------------------------
    Total:                    9 630       52       99

command line: [2]
    -------------------------------------------------
    Total:

dl7M_tln.a: [3]
    exit.o                        4
    low_level_init.o              4
    -------------------------------------------------
    Total:                        8

rt7M_tl.a: [4]
    ABImemclr4.o                  6
    ABImemcpy_unaligned.o        86
    ABImemset48.o                50
    cexit.o                      10
    cmain.o                      26
    copy_init3.o                 44
    cstartup_M.o                 12
    data_init.o                  40
    zero_init3.o                 64
    -------------------------------------------------
    Total:                      338

shb_l.a: [5]
    exit.o                       20
    -------------------------------------------------
    Total:                       20

    Gaps                         10
    Linker created                        38    1 024
-----------------------------------------------------
    Grand Total:             10 006       90    1 123


*******************************************************************************
*** ENTRY LIST
***

Entry                      Address   Size  Type      Object
-----                      -------   ----  ----      ------
.iar.init_table$$Base   0x080025d0          --   Gb  - Linker created -
.iar.init_table$$Limit  0x080025f4          --   Gb  - Linker created -
?main                   0x080025f5         Code  Gb  cmain.o [4]
AHBPrescTable           0x08002648   0x10  Data  Gb  system_stm32f1xx.o [1]
APBPrescTable           0x08002680    0x8  Data  Gb  system_stm32f1xx.o [1]
BusFault_Handler        0x08002553    0x2  Code  Gb  stm32f1xx_it.o [1]
CSTACK$$Base            0x20000010          --   Gb  - Linker created -
CSTACK$$Limit           0x20000410          --   Gb  - Linker created -
DebugMon_Handler        0x08002559    0x2  Code  Gb  stm32f1xx_it.o [1]
Error_Handler           0x08001d23    0x2  Code  Gb  main.o [1]
HAL_DMA_Abort_IT        0x08001d25  0x1be  Code  Gb  stm32f1xx_hal_dma.o [1]
HAL_DMA_GetState        0x08001f1d    0x6  Code  Gb  stm32f1xx_hal_dma.o [1]
HAL_GPIO_Init           0x08001f2d  0x2d2  Code  Gb  stm32f1xx_hal_gpio.o [1]
HAL_GetTick             0x080023ff    0x6  Code  Wk  stm32f1xx_hal.o [1]
HAL_I2C_AbortCpltCallback
                        0x08000767    0x2  Code  Wk  stm32f1xx_hal_i2c.o [1]
HAL_I2C_AddrCallback    0x0800075d    0x2  Code  Wk  stm32f1xx_hal_i2c.o [1]
HAL_I2C_ER_IRQHandler   0x0800066d   0xec  Code  Gb  stm32f1xx_hal_i2c.o [1]
HAL_I2C_EV_IRQHandler   0x080004d9  0x194  Code  Gb  stm32f1xx_hal_i2c.o [1]
HAL_I2C_ErrorCallback   0x08000765    0x2  Code  Wk  stm32f1xx_hal_i2c.o [1]
HAL_I2C_Init            0x08000131  0x1c4  Code  Gb  stm32f1xx_hal_i2c.o [1]
HAL_I2C_ListenCpltCallback
                        0x0800075f    0x2  Code  Wk  stm32f1xx_hal_i2c.o [1]
HAL_I2C_MasterRxCpltCallback
                        0x08001d21    0x2  Code  Gb  main.o [1]
HAL_I2C_MasterTxCpltCallback
                        0x08001cf7   0x12  Code  Gb  main.o [1]
HAL_I2C_Master_Receive_IT
                        0x080003d1   0xe8  Code  Gb  stm32f1xx_hal_i2c.o [1]
HAL_I2C_Master_Transmit_IT
                        0x080002f5   0xdc  Code  Gb  stm32f1xx_hal_i2c.o [1]
HAL_I2C_MemRxCpltCallback
                        0x08000763    0x2  Code  Wk  stm32f1xx_hal_i2c.o [1]
HAL_I2C_MemTxCpltCallback
                        0x08000761    0x2  Code  Wk  stm32f1xx_hal_i2c.o [1]
HAL_I2C_MspInit         0x08001459   0x92  Code  Gb  stm32f1xx_hal_msp.o [1]
HAL_I2C_SlaveRxCpltCallback
                        0x0800075b    0x2  Code  Wk  stm32f1xx_hal_i2c.o [1]
HAL_I2C_SlaveTxCpltCallback
                        0x08000759    0x2  Code  Wk  stm32f1xx_hal_i2c.o [1]
HAL_IncTick             0x080023ef   0x10  Code  Wk  stm32f1xx_hal.o [1]
HAL_Init                0x0800238d   0x22  Code  Gb  stm32f1xx_hal.o [1]
HAL_InitTick            0x080023af   0x40  Code  Wk  stm32f1xx_hal.o [1]
HAL_MspInit             0x08001411   0x48  Code  Gb  stm32f1xx_hal_msp.o [1]
HAL_NVIC_EnableIRQ      0x08002351    0xe  Code  Gb  stm32f1xx_hal_cortex.o [1]
HAL_NVIC_SetPriority    0x0800232b   0x26  Code  Gb  stm32f1xx_hal_cortex.o [1]
HAL_NVIC_SetPriorityGrouping
                        0x0800231f    0xc  Code  Gb  stm32f1xx_hal_cortex.o [1]
HAL_RCC_ClockConfig     0x08001981  0x16e  Code  Gb  stm32f1xx_hal_rcc.o [1]
HAL_RCC_GetHCLKFreq     0x08001b67    0x6  Code  Gb  stm32f1xx_hal_rcc.o [1]
HAL_RCC_GetPCLK1Freq    0x08001b6d   0x16  Code  Gb  stm32f1xx_hal_rcc.o [1]
HAL_RCC_GetSysClockFreq
                        0x08001aef   0x78  Code  Gb  stm32f1xx_hal_rcc.o [1]
HAL_RCC_OscConfig       0x08001501  0x480  Code  Gb  stm32f1xx_hal_rcc.o [1]
HAL_SYSTICK_Config      0x0800235f    0xc  Code  Gb  stm32f1xx_hal_cortex.o [1]
HardFault_Handler       0x0800254f    0x2  Code  Gb  stm32f1xx_it.o [1]
I2C1_ER_IRQHandler      0x0800256f    0xa  Code  Gb  stm32f1xx_it.o [1]
I2C1_EV_IRQHandler      0x08002565    0xa  Code  Gb  stm32f1xx_it.o [1]
I2C_ConvertOtherXferOptions
                        0x080013f5   0x1c  Code  Lc  stm32f1xx_hal_i2c.o [1]
I2C_DMAAbort            0x08001355   0xa0  Code  Lc  stm32f1xx_hal_i2c.o [1]
I2C_ITError             0x080011d7  0x178  Code  Lc  stm32f1xx_hal_i2c.o [1]
I2C_MasterReceive_BTF   0x08000a0f  0x128  Code  Lc  stm32f1xx_hal_i2c.o [1]
I2C_MasterReceive_RXNE  0x08000967   0xa8  Code  Lc  stm32f1xx_hal_i2c.o [1]
I2C_MasterTransmit_BTF  0x080008c1   0xa4  Code  Lc  stm32f1xx_hal_i2c.o [1]
I2C_MasterTransmit_TXE  0x08000769  0x158  Code  Lc  stm32f1xx_hal_i2c.o [1]
I2C_Master_ADD10        0x08000be9   0x32  Code  Lc  stm32f1xx_hal_i2c.o [1]
I2C_Master_ADDR         0x08000c1b  0x256  Code  Lc  stm32f1xx_hal_i2c.o [1]
I2C_Master_SB           0x08000b37   0xb2  Code  Lc  stm32f1xx_hal_i2c.o [1]
I2C_SlaveReceive_BTF    0x08000f27   0x1c  Code  Lc  stm32f1xx_hal_i2c.o [1]
I2C_SlaveReceive_RXNE   0x08000edb   0x4c  Code  Lc  stm32f1xx_hal_i2c.o [1]
I2C_SlaveTransmit_BTF   0x08000ebf   0x1c  Code  Lc  stm32f1xx_hal_i2c.o [1]
I2C_SlaveTransmit_TXE   0x08000e73   0x4c  Code  Lc  stm32f1xx_hal_i2c.o [1]
I2C_Slave_ADDR          0x08000f43   0x5c  Code  Lc  stm32f1xx_hal_i2c.o [1]
I2C_Slave_AF            0x08001133   0xa4  Code  Lc  stm32f1xx_hal_i2c.o [1]
I2C_Slave_STOPF         0x08000f9f  0x194  Code  Lc  stm32f1xx_hal_i2c.o [1]
MX_GPIO_Init            0x08001cc1   0x36  Code  Lc  main.o [1]
MX_I2C1_Init            0x08001c77   0x4a  Code  Lc  main.o [1]
MemManage_Handler       0x08002551    0x2  Code  Gb  stm32f1xx_it.o [1]
NMI_Handler             0x0800254d    0x2  Code  Gb  stm32f1xx_it.o [1]
NVIC_EncodePriority     0x080022b1   0x3e  Code  Lc  stm32f1xx_hal_cortex.o [1]
PendSV_Handler          0x0800255b    0x2  Code  Gb  stm32f1xx_it.o [1]
RCC_Delay               0x08001b83   0x26  Code  Lc  stm32f1xx_hal_rcc.o [1]
Region$$Table$$Base     0x080025d0          --   Gb  - Linker created -
Region$$Table$$Limit    0x080025f4          --   Gb  - Linker created -
SVC_Handler             0x08002557    0x2  Code  Gb  stm32f1xx_it.o [1]
SysTick_Config          0x080022ef   0x30  Code  Lc  stm32f1xx_hal_cortex.o [1]
SysTick_Handler         0x0800255d    0x8  Code  Gb  stm32f1xx_it.o [1]
SystemClock_Config      0x08001c11   0x66  Code  Gb  main.o [1]
SystemCoreClock         0x20000004    0x4  Data  Gb  system_stm32f1xx.o [1]
SystemInit              0x080024a5   0x4e  Code  Gb  system_stm32f1xx.o [1]
UsageFault_Handler      0x08002555    0x2  Code  Gb  stm32f1xx_it.o [1]
__NVIC_EnableIRQ        0x08002271   0x1a  Code  Lc  stm32f1xx_hal_cortex.o [1]
__NVIC_GetPriorityGrouping
                        0x08002267    0xa  Code  Lc  stm32f1xx_hal_cortex.o [1]
__NVIC_SetPriority      0x0800228b   0x26  Code  Lc  stm32f1xx_hal_cortex.o [1]
__NVIC_SetPriorityGrouping
                        0x08002249   0x1e  Code  Lc  stm32f1xx_hal_cortex.o [1]
__aeabi_memclr4         0x08001f25         Code  Gb  ABImemclr4.o [4]
__cmain                 0x080025f5         Code  Gb  cmain.o [4]
__exit                  0x08002625   0x14  Code  Gb  exit.o [5]
__iar_Memset4_word      0x08002471         Code  Gb  ABImemset48.o [4]
__iar_Memset8_word      0x08002471         Code  Gb  ABImemset48.o [4]
__iar_copy_init3        0x0800257d   0x2c  Code  Gb  copy_init3.o [4]
__iar_data_init3        0x080025a9   0x28  Code  Gb  data_init.o [4]
__iar_program_start     0x08002669         Code  Gb  cstartup_M.o [4]
__iar_unaligned___aeabi_memcpy4
                        0x08002419         Code  Gb  ABImemcpy_unaligned.o [4]
__iar_unaligned___aeabi_memcpy8
                        0x08002419         Code  Gb  ABImemcpy_unaligned.o [4]
__iar_zero_init3        0x0800250d   0x40  Code  Gb  zero_init3.o [4]
__low_level_init        0x0800260f    0x4  Code  Gb  low_level_init.o [3]
__vector_table          0x08000000         Data  Gb  startup_stm32f103xe.o [1]
_call_main              0x08002601         Code  Gb  cmain.o [4]
_exit                   0x08002619         Code  Gb  cexit.o [4]
_main                   0x0800260b         Code  Gb  cmain.o [4]
exit                    0x08002613    0x4  Code  Gb  exit.o [3]
hi2c1                   0x20000410   0x54  Data  Gb  main.o [1]
main                    0x08001bf1   0x20  Code  Gb  main.o [1]
regAddress              0x20000008    0x1  Data  Gb  main.o [1]
regData                 0x20000468    0x1  Data  Gb  main.o [1]
uwTick                  0x20000464    0x4  Data  Gb  stm32f1xx_hal.o [1]
uwTickFreq              0x20000009    0x1  Data  Gb  stm32f1xx_hal.o [1]
uwTickPrio              0x20000000    0x4  Data  Gb  stm32f1xx_hal.o [1]


[1] = D:\Projects\MicroTechnics\Projects_site\MT_I2C_Example\EWARM\MT_I2C_Example\Obj
[2] = command line
[3] = dl7M_tln.a
[4] = rt7M_tl.a
[5] = shb_l.a

  10 006 bytes of readonly  code memory
      90 bytes of readonly  data memory
   1 123 bytes of readwrite data memory

Errors: none
Warnings: none
